:100000000C9469000C9491000C9491000C94910054
:100010000C9491000C9491000C9491000C9491001C
:100020000C9491000C9491000C9491000C94920B00
:100030000C9491000C9491000C9491000C949100FC
:100040000C9410130C9491000C9435160C946716B4
:100050000C9491000C9491000C9491000C949100DC
:100060000C94720A0C949100000000090003020035
:10007000000405080000000000000000000000016E
:10008000020408102040800102040810200102042C
:100090000810204080400404040404040404020204
:1000A000020202020303030303030202030000002F
:1000B0000023002600290000000000250028002B56
:1000C0000000000000240027002A000074036309D8
:1000D000971611241FBECFEFD8E0DEBFCDBF12E0D0
:1000E000A0E0B1E0EEEAF0E302C005900D92A0348A
:1000F000B107D9F725E0A0E4B2E001C01D92A73016
:10010000B207E1F710E0C9E6D0E004C02197FE0194
:100110000E942018C636D107C9F70E94B3170C9465
:1001200055180C940000862F642F0C947D14FC014C
:1001300081890E94E71421E0892B09F420E0822FB5
:100140000895FC01DB0182E891E09183808312969F
:100150004D915D916D917C9115974283538364839A
:10016000758316968D919C91179797838683189621
:100170008C911897808719964D915D916D917C9126
:100180001C9741875287638774871D964D915D91B7
:100190006D917C915097458756876787708B5196F4
:1001A0008C915197818B88E891E09183808352965E
:1001B0008C91828B0895CF92DF92EF92FF920F93F2
:1001C0001F93CF93DF9326E040E855E260E070E0B4
:1001D0008AE694E00E94E3150E947D0D83E793E098
:1001E0000E94CB088BEF92E00E940D088BEF92E00B
:1001F0000E9412078BEF92E00E945D0709EF11E069
:10020000C3E6D2E08DEFC82E81E0D82E7801F70149
:1002100061917F0170E0CE010E94E50665E070E02B
:10022000CE010E944F061A8A6396CE14DF0479F736
:1002300063E070E080E692E00E94E70C60910C01C0
:1002400070E080E692E00E94220D80E592E00E943C
:10025000660F80E492E00E94660F61E084E00E94F5
:100260007D1461E08EE00E947D1461E08FE00E94C9
:100270007D1461E085E00E947D1461E086E00E94CB
:100280007D1461E089E00E947D1461E081E10E94BB
:100290007D1461E082E00E947D1462E0F8018191AA
:1002A0008F010E947D14F1E00E3F1F07B1F761E05E
:1002B00084E00E94B91470E060E085E00E94F713CA
:1002C00070E060E086E00E94F71370E060E089E093
:1002D0000E94F71360E081E10E94B91460E082E0BF
:1002E0000E94B9148FE580936A0380936B03809317
:1002F0006C0380936D0380936E0380936F038093F0
:10030000700380937103DF91CF911F910F91FF9044
:10031000EF90DF90CF9008950F931F93CF93DF93CB
:100320008B01EA01BC0185E00E94F713B80186E069
:100330000E94F713BE0189E0DF91CF911F910F91C9
:100340000C94F71350E040E070E060E090E080E053
:100350000C948C01813041F028F0823069F08330B8
:1003600091F008950C94A20150E040E070E060E04C
:100370008FEF90E00C948C0150E040E06FEF70E064
:1003800090E080E0F7CF4FEF50E070E060E0F8CF12
:100390008BEF92E00E945D0740E062E08BEF92E01D
:1003A0000E946B076EE071E08BEF92E00E940017F5
:1003B00041E060E08BEF92E00E946B076AE673E039
:1003C0008BEF92E00E9400178BEF92E00C941707DE
:1003D0000E94451861E0892B09F04CC086E00E941C
:1003E000B9148BEF92E00E945D0740E065E08BEF6F
:1003F00092E00E946B0764E371E08BEF92E00E9451
:10040000001741E062E08BEF92E00E946B076BE324
:1004100071E08BEF92E00E94001761E084E00E949F
:10042000B9148091080180930A0160910B0170E07A
:1004300080E692E00E94220D68EB7BE080E090E095
:100440000E948B1360E086E00E94B9148BEF92E06B
:100450000E945D078BEF92E00E94170740E060E08A
:100460008BEF92E00E946B0767E471E08BEF92E004
:100470000C94001785E00E94B9148BEF92E00E9463
:100480005D0740E065E08BEF92E00E946B0764E35C
:1004900071E08BEF92E00E94001741E065E08BEF86
:1004A00092E00E946B0768E571E08BEF92E00E949A
:1004B000001768EB7BE080E090E00E948B1360E027
:1004C00085E00C94B914AF92BF92CF92DF92EF9275
:1004D000FF920F931F93CF93DF937C01FC01019058
:1004E0000020E9F731978F01081B190B680120E103
:1004F000C21AD10880E1A82EB12C8091590380172F
:100500001106A1F041E060E08BEF92E00E946B07E2
:1005100001311105C4F4B7018BEF92E00E9400177E
:1005200068EB7BE080E090E00E948B13109259030F
:10053000DF91CF911F910F91FF90EF90DF90CF90BF
:10054000BF90AF9008958091590390E0E701C80FE4
:10055000D91F8C159D052CF520915903822F90E011
:100560000F96AE014E195F098417950734F0699113
:100570008BEF92E00E940817EFCF211106C06CEDBF
:1005800075E080E090E00E948B136CE271E080E007
:1005900090E00E948B13809159038F5F80935903E1
:1005A000ACCFCE018E199F098017910734F4699161
:1005B0008BEF92E00E940817F4CFD0E0C0E080916A
:1005C00059039801281B3109C9019501281B390BD2
:1005D0002C173D07D4F260E28BEF92E00E940817DF
:1005E0002196EDCFCF93C82F8BEF92E00E945D074D
:1005F0008BEF92E00E94170740E0CA3009F443C035
:1006000060E08BEF92E00E946B0760E671E08BEF99
:1006100092E00E9400174AE050E06C2F8BEF92E0CE
:100620000E946817C230E9F108F5609106017091E7
:100630000701C13019F180E393E00E9463028BEF60
:1006400092E00E945D0780910A01843020F48BEFD4
:1006500092E00E941207E0E3F3E088E593E020E2F5
:1006600021938E179F07E1F7CF910895C330F1F0E2
:100670006091000170910101C430E9F680E393E0DC
:100680000E944E18D8CF61E08BEF92E00E946B077A
:100690006FE671E08BEF92E00E94001768E073E074
:1006A000EDCF6091040170910501E8CF60910201E6
:1006B00070910301E3CFDC01FB019C9180819813D1
:1006C00011C011969C911197818198130BC01296BD
:1006D0009C9112978281981305C081E013962C910A
:1006E0009381291380E008950F931F93CF9322E005
:1006F00040E160910D018BEF92E00E94ED0688EEE3
:1007000092E00E94D806E8EEF2E008E811E01183DA
:100710000083C1E0C28B85ED92E00E94D806E5ED32
:10072000F2E011830083C28B82EC92E00E94D80633
:10073000E2ECF2E011830083C28B8FEA92E00E9428
:10074000D806EFEAF2E011830083C28B68EE72E014
:1007500083E692E00E94A10065ED72E086E792E0F8
:100760000E94A10062EC72E089E892E00E94A10080
:100770006FEA72E08CE992E00E94A10080E692E0CC
:100780000E944D0C40E16EE080E592E00E94430E35
:1007900040E16FE080E492E0CF911F910F910C94C3
:1007A000430EFF920F931F93CF93DF9390910A0113
:1007B0008091090198130E94C801C3E6D2E010E0BD
:1007C00000E0CE010E946B06888582FF22C0CE0128
:1007D0000E94D4069A8989131CC060916903F801AC
:1007E000EC50FE4FF080E62FF0E0E659FC4FF0822F
:1007F00041E08BEF92E00E946B076F2D8BEF92E050
:100800000E94A307809169038F5F809369030E9410
:10081000C8010F5F1F4F63960430110591F6809158
:100820006903883031F563E271E08AE693E00E9463
:10083000E801109269038FE580936A0380936B034C
:1008400080936C0380936D0380936E0380936F039A
:10085000809370038093710390910A018091080145
:10086000981739F0DF91CF911F910F91FF900C9461
:10087000C801DF91CF911F910F91FF9008950F93C1
:100880001F930E945A1300915C0310915D03209105
:100890005E0330915F03601B710B820B930B603121
:1008A00077428105910578F080915B0381110BC03F
:1008B000109265031092660310926703109268030A
:1008C00081E080935B0380E592E00E94991290E0C2
:1008D000909363038093620380E592E00E94B30DDE
:1008E000282F30E03093610320936003209162034E
:1008F00030916303232B09F452C0882309F44FC0BD
:100900008091530280936503809154028093660323
:10091000809155028093670380915602809368030B
:1009200010925B0380E592E00E94C91280E592E09C
:100930000E940C130E945A1360935C0370935D0332
:1009400080935E0390935F0365E673E08FE191E02F
:100950000E945B038093640381110DC081E00E94BB
:10096000AA0168EB7BE080E090E00E948B131F916E
:100970000F910C94A2018130A9F482E00E94AA0197
:1009800068EB7BE080E090E00E948B130E94A20164
:1009900080910A01833019F484E080930A011F9149
:1009A0000F9108958230D9F783E00E94AA0168E58B
:1009B00072E080E090E0D9CFCF938AE694E00E9485
:1009C000101518161906B4F48AE694E00E942A1548
:1009D00080935803883609F46BC0ECF4833309F430
:1009E00072C054F4813309F468C00CF06AC08432D8
:1009F00009F493C0CF910895823609F452C024F4CB
:100A00008433C1F784E05AC0833609F478C087364E
:100A100089F782E043C0823709F43FC034F58F364E
:100A200009F441C0803709F441C08D3619F764E6F6
:100A300070E080E090E00E948B13C0E08AE694E0D2
:100A40000E941015181619060CF05CC08AE694E096
:100A50000E942A1580930703843281F3EC2FF0E083
:100A6000E85FFC4F8083CF5FE9CF853771F144F4B5
:100A700060E0833709F0BECF84E0CF910C94B914C5
:100A8000863781F160910B01873709F0B3CF70E0B1
:100A900080E692E0CF910C94220D81E0CF910C94EE
:100AA000AA0183E0FBCFCF910C94A20161E0E4CFD7
:100AB00080910A01CF910C94F20281E080930A01A7
:100AC00099CF82E0FBCF83E0F9CF61E081E10E9422
:100AD000B91468EB7BE080E090E00E948B1360E04B
:100AE00081E1CBCF61E082E00E94B91468EB7BE04A
:100AF00080E090E00E948B1360E082E0BECF6091C6
:100B00000C01C5CF8AE00E94F202E8E0F3E0119206
:100B100083E0E033F807D9F76DCF62E370E080E05F
:100B200090E00E948B134AE050E060910A018AE64F
:100B300094E0CF910C94681760910A0180910901AB
:100B4000681731F04AE050E08AE694E00E946817A6
:100B500080910A0180930901813020F0843058F19E
:100B6000863090F18AE00E94E714892B79F484E0C2
:100B70000E94E714019769F560E084E00E94B914CF
:100B800060ED77E080E090E00E948B130E94DC042F
:100B900042E069E083E793E00E945D0983E793E028
:100BA0000E94160880935A0390910A01811116C081
:100BB000913089F508958BEF92E00E945D078BEFED
:100BC00092E00E941207CECF8BEF92E00E941707AF
:100BD000C9CF80910A010E94F202D8CF8130D9F4A6
:100BE000913019F482E080930A0161E081E10E9472
:100BF000B91460E777E180E090E00E948B1360E039
:100C000081E10E94B9146CE271E080E090E00E9402
:100C10008B1310925A0380910A0190915A039230DB
:100C200019F08230E1F40895823019F483E0809362
:100C30000A0161E082E00E94B91460E777E180E098
:100C400090E00E948B1360E082E00E94B9146CE295
:100C500071E080E090E00E948B1310925A03809123
:100C60000A01833010F00E943F0480910A01843011
:100C700031F48BEF92E00E9417070C94D103089592
:100C8000FC0182E891E091838083128213821482B6
:100C900015828AE090E09783868310860895FC0190
:100CA000778366830895CF93DF93EC011886E881FC
:100CB000F9810190F081E02D0995882319F088854C
:100CC000836088870E945A136A837B838C839D8309
:100CD000DF91CF910895CF92DF92EF92FF920F9321
:100CE0001F93CF93DF93EC0188858B7F8887E88102
:100CF000F9810190F081E02DCE010995182F8885AA
:100D0000869581701817B9F00E945A136A837B8305
:100D10008C839D83888592E089278887888582FBDC
:100D2000882780F9DF91CF911F910F91FF90EF906D
:100D3000DF90CF9008950E945A13CA80DB80EC8028
:100D4000FD80AB01BC014C195D096E097F098E81E4
:100D50009F81B0E0A0E0481759076A077B07F0F2CF
:100D6000888581701817D1F20E945A136A837B8399
:100D70008C839D83888591E08927846088870E9481
:100D80005A1309851A852B853C85601B710B820BD4
:100D9000930B6D877E878F87988B0E945A13698784
:100DA0007A878B879C87BACFFC01808581700895F4
:100DB000CF93DF93EC010E94400681E092E099839B
:100DC0008883198ADF91CF910895FC01618B0C947F
:100DD000530690E080E008950895FC01138212828A
:100DE00089E092E091838083648341872287138620
:100DF00008950F931F93CF938C01C62FFC0164813C
:100E000083E793E00E94DD08F80163856C2B83E79C
:100E100093E00E946F0883E793E0CF911F910F91B9
:100E20000C946009FC01138660E00C94F90628E03C
:100E3000FC01238760E00C94F9060F931F93CF9376
:100E40008C01C62F64600E94F90681E090E00E9448
:100E5000C4136C2F6B7FC8010E94F90682E390E0F7
:100E6000CF911F910F910C94C4131F93CF93DF93D5
:100E7000EC01162F0E94F906612FCE01DF91CF9170
:100E80001F910C941D070F931F93CF93DF938C0139
:100E9000D62FC42F607F642B0E94350780E1D89F36
:100EA000B00111246C2BC801DF91CF911F910F91DC
:100EB0000C94350740E00C94430761E00E945A0708
:100EC00080ED97E00C94C41362E00E945A0780ED15
:100ED00097E00C94C413CF93DF93CDB7DEB7289778
:100EE0000FB6F894DEBF0FBECDBF28E0ECE2F1E014
:100EF000DE01119601900D922A95E1F7FC01208503
:100F0000241710F44FEF420F50E0440F551F21E01B
:100F100030E02C0F3D1F420F531FFA012081620F5A
:100F2000606828960FB6F894DEBF0FBECDBFDF9184
:100F3000CF910C945A07FC016681262F24602683EA
:100F40006C600C945A0741E00E94430781E090E0F6
:100F50000895CF93DF93EC01423018F08D818860C3
:100F60008D834887222329F0413019F48D818460D4
:100F70008D8362E370E080E090E00E948B136B85CC
:100F8000CE010E94F90668EE73E080E090E00E94D6
:100F90008B1360E3CE010E94350784E991E10E9442
:100FA000C41360E3CE010E94350784E991E10E94F9
:100FB000C41360E3CE010E94350786E990E00E94E9
:100FC000C41360E2CE010E9435076D816062CE01DC
:100FD0000E945A0784E08E83CE010E949B07CE01B7
:100FE0000E945D0782E08F8366E0CE010E945A076F
:100FF000CE01DF91CF910C946407CF93DF93EC0186
:1010000083E793E00E94CB081D8220E04A85698532
:10101000CE01DF91CF910C94A9070C94FD0780912C
:10102000A7039091A803891B990B08959091A80399
:101030008091A7032FEF3FEF981748F4E92FF0E0D6
:10104000E755FC4F208130E09F5F9093A803C901D2
:101050000895E091A8038091A703E81730F4F0E029
:10106000E755FC4F808190E008958FEF9FEF089542
:101070000895CF93DF93EC01E0917F03F09180031B
:101080003097F1F09091A8038091A7039817C0F0D2
:1010900090E0292F30E02617370754F4DE01A20F25
:1010A000B31F4C9127553C4FD9014C939F5FF1CF13
:1010B0001092A8036093A703CB01DF91CF9109940D
:1010C000DF91CF910895E0918103F09182033097F1
:1010D00029F0109285031092840309940895CF9308
:1010E000DF931F92CDB7DEB769832091830322235C
:1010F000F9F020918403203258F021E030E0FC0127
:101100003383228390E080E00F90DF91CF910895A8
:1011100080918503E82FF0E0EA57FC4F9981908396
:101120008F5F809385038093840381E090E0ECCF10
:1011300061E0CE0101960E94310AF7CFCF92DF9293
:10114000EF92FF920F931F93CF93DF937C01CB011C
:101150008A0120918303222389F0EB016B01C40EE5
:10116000D51ECC15DD0569F06991D701ED91FC9193
:101170000190F081E02DC7010995F3CF642F0E9403
:10118000310AC801DF91CF911F910F91FF90EF902D
:10119000DF90CF9008951092A8031092A7031092A9
:1011A0008503109284030E94740983E698E00E94EC
:1011B0005D0A89E398E00C94580A81E080938303E8
:1011C0006093A603109285031092840308950F93F1
:1011D000062F21E04091840366E873E08091A60326
:1011E0000E94DA09109285031092840310928303FF
:1011F0000F9108954F925F926F927F92AF92BF923C
:10120000CF92EF92FF920F931F93CF93DF935C01E6
:10121000F62ED42F28013901EE2019F10E94DD08A5
:10122000CE2DC43008F0C3E0C150B8F028E0C29F12
:10123000C0011124A301920104C05695479537952A
:1012400027958A95D2F7B901D501ED91FC910190CE
:10125000F081E02DC5010995E7CF60E0C5010E944E
:10126000E7084D2FD13208F040E22C2D69EA73E0F7
:101270008F2D0E9492091092A8038093A703DF91FB
:10128000CF911F910F91FF90EF90CF90BF90AF90B3
:101290007F906F905F904F900895CF92EF920F9351
:1012A0001F93C22EE12C00E010E098010E94FA0882
:1012B0001F910F91EF90CF90089521E00C944D096C
:1012C00061E00C94E708E3E7F3E01382128288EE12
:1012D00093E0A0E0B0E084839583A683B78385E1A3
:1012E00092E09183808308951092360481E0809388
:1012F00034041092330461E082E10E94B91461E089
:1013000083E10E94B914E9EBF0E080818E7F808355
:1013100080818D7F808380E28093B80085E4809314
:10132000BC000895413208F043C0909136049111F9
:10133000FCCF91E090933604209334042FEF209358
:10134000C90310920E04240F20930D0490933504CA
:1013500090913504880F892B809335048091330454
:10136000813009F510923304809135048093BB00DD
:101370008091BC0083FDF8CF85EC8093BC00809108
:1013800036048130E1F380910E04841710F440910B
:101390000E04AFE0B4E0962FFB018E2F891B84175B
:1013A00020F0842F089585EEE8CF8D918193F5CFBD
:1013B00040E0F7CF0F93413208F04BC090913604D4
:1013C0009111FCCF92E090933604009334049FEF88
:1013D0009093C90310920E0440930D04362FAFE092
:1013E000B4E0FB019E2F931B941770F1109235040B
:1013F00090913504880F892B8093350480913304B4
:10140000813029F510923304809135048093BB001C
:101410008091BC0083FDF8CF85EC8093BC00222333
:1014200021F0809136048230D1F38091C9038F3F3F
:1014300091F08091C903803281F08091C90380339B
:1014400071F084E00F91089591919D93CBCF85EE3B
:10145000E4CF81E0F7CF80E0F5CF82E0F3CF83E007
:10146000F1CF2091EB03260F3327331F21323105B3
:10147000ECF420913604FC0190E080E0243069F027
:1014800082E00895A091EB032191AC0143515C4FA0
:10149000A40FB52FB11D2C930196861798F3809158
:1014A000EB03680F6093EB0380E0089581E00895FB
:1014B0009093300480932F04089590933204809386
:1014C0003104089585ED8093BC008091BC0084FDBB
:1014D000FCCF10923604089585EC8093BC001092E6
:1014E000360408951F920F920FB60F9211242F9376
:1014F0003F934F935F936F937F938F939F93AF939C
:10150000BF93EF93FF938091B900887F803609F4F1
:101510004CC008F03FC0883209F4A8C018F58031EB
:1015200009F49CC0B8F4882309F4F9C0883009F4A0
:1015300095C0FF91EF91BF91AF919F918F917F9156
:101540006F915F914F913F912F910F900FBE0F9030
:101550001F901895883109F489C0803251F7809323
:10156000C90315C0803409F49EC048F48033B9F330
:101570008833F9F68093C9030E946C0ADACF80356C
:1015800009F485C0883509F496C0883491F60E9424
:10159000620ACFCF883909F48CC038F5883729F032
:1015A00050F4883611F0803721F683E080933604BA
:1015B0001092CA0357C0883809F47BC0803919F0EB
:1015C000803809F0B6CF8091CA03803208F071C02C
:1015D000E091CA0381E08E0F8093CA038091BB0023
:1015E000F0E0E553FC4F80833DC0803B39F0E0F4F0
:1015F000803A09F479C0883A09F09BCF84E080935F
:1016000036041092EC031092EB03E0913104F09158
:10161000320409958091EB0381110FC081E0809322
:10162000EB031092ED0309C0803C09F476C0883CBE
:1016300009F473C0883B09F07CCFE091EC0381E0B2
:101640008E0F8093EC03F0E0E351FC4F8081809398
:10165000BB009091EC038091EB0329C0809135048D
:101660008093BB0085EC8093BC0063CF90910E0407
:1016700080910D04981758F5E0910E0481E08E0FCB
:1016800080930E04F0E0E15FFB4F8081E9CFE091B1
:101690000E0481E08E0F80930E048091BB00F0E079
:1016A000E15FFB4F808390910E0480910D049817A9
:1016B000C8F285E8D8CFE0910E0481E08E0F8093C8
:1016C0000E048091BB00F0E0E15FFB4F80838091CE
:1016D000340481115CCF81E08093330484EA8093E9
:1016E000BC001092360425CF0E946C0A8091CA0378
:1016F000803230F4E091CA03F0E0E553FC4F1082F1
:101700006091CA0370E0E0912F04F09130048BECFB
:1017100093E009951092CA030CCF85ECE0CF1092AC
:10172000C90335CF1F920F920FB60F9211242F933A
:101730003F934F935F936F937F938F939F93AF9359
:10174000BF93EF93FF938091380487FF27C01092D7
:10175000850010928400809138048F5F8093380454
:1017600080913804082E000C990B2091370428171B
:10177000190629F024F0809138048C30DCF1809136
:10178000840090918500049680329E4408F47BC0CA
:101790008091840090918500049677C080913804F0
:1017A000082E000C990B209137042817190699F27E
:1017B00094F2E09138048E2FEE0F990BFC01EE0F9E
:1017C000FF1FE80FF91FE75CFB4F808186FFC3CF47
:1017D000E09138048E2FEE0F990BFC01EE0FFF1FE6
:1017E000E80FF91FE75CFB4F808160E08F730E9478
:1017F000B914B1CF2091840030918500E091380474
:101800008E2FEE0F990BFC01EE0FFF1FE80FF91F53
:10181000E75CFB4F81819281820F931F9093890037
:1018200080938800E09138048E2FEE0F990BFC0115
:10183000EE0FFF1FE80FF91FE75CFB4F808186FF6B
:1018400011C0E09138048E2FEE0F990BFC01EE0FC2
:10185000FF1FE80FF91FE75CFB4F808161E08F738A
:101860000E94B914FF91EF91BF91AF919F918F9119
:101870007F916F915F914F913F912F910F900FBE8C
:101880000F901F90189580E29EE4909389008093BA
:1018900088008FEF80933804E5CFFC0190913704E6
:1018A0009C3098F481E0890F809337049083892FCE
:1018B00090E0FC01EE0FFF1FE80FF91FE75CFB4F04
:1018C0008CED95E09283818308958FEF8083089556
:1018D000DF92EF92FF920F931F93CF93DF93EC0170
:1018E000D62E7A01890188818C3008F067C061E0CA
:1018F0008D2D0E947D148881282F30E0F901EE0F94
:10190000FF1FE20FF31FE75CFB4F9D2D9F7360816C
:10191000607C692B608320E232E02E193F0937FF9B
:1019200002C02D5F3F4F3595279535952795298323
:1019300020E639E0201B310B37FF02C02D5F3F4FFF
:1019400035952795359527952A832CE0622F0E949F
:10195000D317829FB001112430E020E0AB01420F89
:10196000531FFA01EE0FFF1FE40FF51FE75CFB4F5B
:10197000908196FD16C02F5F3F4F2C30310571F7D7
:1019800081110FC01092800082E08093810010923C
:10199000850010928400B19A80916F0082608093DC
:1019A0006F00E8818E2F90E0FC01EE0FFF1FE80F23
:1019B000F91FE75CFB4F8081806480838881DF9121
:1019C000CF911F910F91FF90EF90DF90089520E647
:1019D00039E040E252E00C94680CDC01EC91EC3010
:1019E00080F511968C91119728E830E0281B310979
:1019F00087FD3395220F331F220F331F62177307A2
:101A000084F012968C9128E532E0281B310987FD7D
:101A10003395220F331F220F331F621773070CF405
:101A20009B014FB7F8948E2F90E022503109FC01B2
:101A3000EE0FFF1FE80FF91FE75CFB4F3283218396
:101A40004FBF0895AF92BF92CF92DF92EF92FF9275
:101A50000F931F93CF93DF93EC01603282E07807FE
:101A60000CF03EC0653B710514F064EB70E08981B9
:101A700048E8A42EB12CA81AB10887FDB394AA0C8B
:101A8000BB1CAA0CBB1C0B2C000CCC08DD0877FF80
:101A900002C070E060E0072E000C880B990B2A81D1
:101AA00008E512E0021B110927FD1395000F111F15
:101AB000000F111F012E000C220B330B3F932F93AD
:101AC0001F930F9314EBE12EF12C00E010E020E0C7
:101AD00030E0A9010E946F170F900F900F900F90A8
:101AE000CE01DF91CF911F910F91FF90EF90DF908A
:101AF000CF90BF90AF900C94ED0CCF93CFB7F894EC
:101B000080916004811127C0E0EAF0E08491E9E867
:101B1000F0E09491E82FF0E0EE0FFF1FEF53FF4F3E
:101B2000A591B491EC91E92321F461E08AE00E944F
:101B3000B91461E08AE00E947D148CB580618CBD8F
:101B40008CB580648CBD61E08DE00E947D1461E005
:101B50008BE00E947D14809160048F5F809360040D
:101B6000CFBFCF910895BC016E5F7F4FDC01ED9137
:101B7000FC910190F081E02D40E0099591E0811108
:101B800090E0892F089520915F04222381F03FB7D0
:101B9000F89420915F04213069F42DB320935D0403
:101BA0004DB320915E04209524232DBB3FBF8CBDF7
:101BB0009DBD089530935D04FACF8EBD00000DB435
:101BC00007FEFDCF8EB5089580915F04882361F0F4
:101BD0009FB7F89420915F0480915D04213019F43F
:101BE0008DBB9FBF08958FBF0895CF92DF92EF9274
:101BF000FF920F931F93CF93DF937C01C42EE901D3
:101C0000D62E6894D7F880E591E00E94C30D60E07D
:101C1000F70186850E94B914CA948D2D0E94DD0DAE
:101C20000023A1F08FEF90E09C0102C0220F331F30
:101C30000A95E2F789018D2D0E94DD0D902F909578
:101C4000288192238023892B888301E0C00FD11D36
:101C50000C1530F48D2D0E94DD0D89930F5FF8CFA8
:101C600080E00E94DD0D888361E0F70186850E9497
:101C7000B914DF91CF911F910F91FF90EF90DF90FA
:101C8000CF900C94E40DFC0187E292E09183808375
:101C90006687478708950F931F93CF93DF93EC01D7
:101CA000062F142F80E591E00E94C30D60E08E8521
:101CB0000E94B914802F0E94DD0D812F0E94DD0D3E
:101CC00061E08E850E94B914DF91CF911F910F9131
:101CD0000C94E40DDF92EF92FF920F931F93CF933A
:101CE000DF937C01C62F042FD22E132F80E591E0C5
:101CF0000E94C30D60E0F70186850E94B9148C2F05
:101D00000E94DD0DCD2DD12F0C0F1D2F111DC017E1
:101D1000D10721F089910E94DD0DF9CF61E0F70133
:101D200086850E94B914DF91CF911F910F91FF908A
:101D3000EF90DF900C94E40D1F93CF93DF93EC01B1
:101D4000162F80E591E00E94C30D60E08E850E9411
:101D5000B914812F80680E94DD0D80E00E94DD0DA6
:101D6000182F61E08E850E94B9140E94E40D812F26
:101D7000DF91CF911F9108950F9341110E94F50DAE
:101D80000F9108950F931F93CF93DF938C01D62F5C
:101D9000C42F0E949C0E482F4C2B6D2FC801DF9141
:101DA000CF911F910F910C944B0E0F931F93CF93D4
:101DB000DF938C01D62FC42F0E949C0EC0954C2F10
:101DC00048236D2FC801DF91CF911F910F910C9483
:101DD0004B0ECF92DF92EF92FF920F931F93CF9310
:101DE000DF93EC016B01142F790140E062E00E9467
:101DF0004B0E44E06AE0CE010E944B0E40E864E1E5
:101E0000CE010E944B0E9601412F62E1CE010E944D
:101E10006A0E43E062E0CE010E944B0E08E813E137
:101E20006AE0CE010E949C0E82FF1BC040E062E08F
:101E3000CE010E944B0E64E4CE010E949C0EF7017D
:101E4000808362E4CE010E949C0EF701818380E0D2
:101E5000DF91CF911F910F91FF90EF90DF90CF9086
:101E6000089501501109E1F683E0F2CF0F931F931B
:101E7000CF938C014FE062E00E944B0EC3E062E31F
:101E800070E080E090E00E948B1362E0C8010E9445
:101E90009C0E84FF02C0C15091F7CF911F910F910A
:101EA0000895CF93DF93EC0168E20E949C0E982F77
:101EB0009370933041F0482F436068E2CE01DF9188
:101EC000CF910C944B0EDF91CF910895CF93DF9378
:101ED000EC0161E08E850E947D1461E08E850E9498
:101EE000B9148F858F3F09F451C060E00E947D14C2
:101EF0008F850E94E714892B09F048C061E08F8527
:101F00000E947D1460E08F850E94B91482E090E009
:101F10000E94C41361E08F850E94B91462E370E0EF
:101F200080E090E00E948B1340E064E2CE010E94CA
:101F30004B0E40E066E2CE010E944B0E46E268E4A2
:101F4000CE010E944B0E40E864E5CE010E944B0E8C
:101F500049EA66E5CE010E944B0E43E068E5CE01FA
:101F60000E944B0E48EE6AE5CE010E944B0E40E403
:101F70006AE2CE010E944B0E4DE362E2CE010E9466
:101F80004B0ECE01DF91CF910C94510FCE010E94E8
:101F9000360FCACF3F924F925F926F927F928F928D
:101FA0009F92AF92BF92CF92DF92EF92FF920F93E8
:101FB0001F93CF93DF9300D0CDB7DEB73C01162F30
:101FC000942E290180E0A114B10411F0F501808163
:101FD000382C329490EF3922380E40E062E0C30191
:101FE0000E944B0E4FE768E0C3010E944B0E40E891
:101FF00064E1C3010E944B0E9201402F62E1C301D4
:102000000E946A0E432D6AE1C3010E944B0E412FCC
:1020100062E0C3010E944B0E1C3029F440E86AE1E3
:10202000C3010E94C20E00ED17E068E0C3010E94E8
:102030009C0E982F992109F07BC080FD03C00150B0
:10204000110999F783E038C0E114F10409F448C09C
:10205000C114D10409F444C064E1C3010E949C0E80
:10206000F6019081981708F45FC08083082D9701CE
:10207000482F62E1C3010E94BC0E68E1C3010E94C7
:102080009C0E8770A114B10411F0F501808313FD3B
:102090004DC0E114F10409F445C0C114D10409F4A0
:1020A00041C09E899923F1F1F60140814130D1F47C
:1020B000843009F047C08FEF0F900F90DF91CF91E0
:1020C0001F910F91FF90EF90DF90CF90BF90AF9056
:1020D0009F908F907F906F905F904F903F9008956A
:1020E00080E0D5CF423070F181112CC042509E016A
:1020F0002F5F3F4FB701C3010E94E90E8111DCCF72
:10210000F6018081E80EF11CF701329790818981F8
:10211000981318C0F1E0EF1AF108F70190818A8155
:10212000981310C080E0C8CF84E0C6CF82E0C4CF4F
:102130006CE0C3010E949C0E182F837109F484CFB8
:1021400081E0BACF87E0B8CF8F92AF92BF92CF92A3
:10215000DF92EF92FF920F931F93AF928C2C570157
:1021600068017901042F9B0140E36CE00E94CA0FD3
:102170000F901F910F91FF90EF90DF90CF90BF9045
:10218000AF908F9008952F923F924F925F926F92EF
:102190007F928F929F92AF92BF92CF92DF92EF92F7
:1021A000FF920F931F93CF93DF93CDB7DEB72D9799
:1021B0000FB6F894DEBF0FBECDBF16E0413508F074
:1021C00045C1342E4B013C0140E86CE10E94D50E24
:1021D00083E98983332029F081E0F40190819530EF
:1021E00008F480E022242394B12C9B2D990F990FA1
:1021F000990FD32CD91AD7FCD12C32E0882319F0AF
:1022000098E89B8333E021E09D2D977009F420E04E
:102210009D2D959595959595290FC9F094E081117F
:1022200093E0291708F4922FEB2DF0E03196E80D9A
:10223000F91D232F4191A1E0B0E0AC0FBD1FA20F0B
:10224000B11D4C932F5F422F431B491798F38823EE
:1022500011F0F8E0DF0E8FE18D150CF082C090E7F1
:102260009A838B819C8189279D8189279E818927DB
:102270008F839E01285F3F4F47E0BE016F5F7F4F16
:10228000C3010E94E90E182F8111E0C01B86E3E014
:10229000EA87DC86CE0107962C0199E09D87CB84E6
:1022A0004C2D4295407F4C0D6AE1C3010E944B0EBC
:1022B000A12CCE010B967C018E01065F1F4F92016F
:1022C0004D85BE016F5F7F4FC3010E94A410182F80
:1022D000823009F065C06CE1C3010E949C0E85FD4F
:1022E000B5C08F7109F480E2282F30E04D2DDD0C50
:1022F000550B421753070CF09DC0D82EE82FE595DB
:10230000E595E595EF5F982F977081E009F480E0FF
:10231000E80F81E090E08C0F9D1F8E0F911DFC0156
:10232000215031092770332781E090E002C0880FE7
:10233000991F2A95E2F79C018081822B80838BCFA5
:1023400085E98983332031F081E0F4019081983070
:1023500008F04BCF80E049CF87E9898326E0B22E91
:10236000F9CF9D2D97709B878D2D859585958595AA
:102370008E5F282F2295207F290F2A8321E091113B
:1023800001C020E0280F2D8744244394512C4C0E8B
:102390005D1E480E511CE9E0E81BEA87DC867FCF12
:1023A000811154C080E2D82E9C8590320CF457CF16
:1023B0008B81883809F040C083E093E0EB2DF0E09A
:1023C0003196E80DF91D980FA1E0B0E0AC0FBD1FEC
:1023D000A80FB11D2C9121938F5F8913F5CFBA847B
:1023E000E3E0BE124DC08B8581114AC09E012D5F76
:1023F0003F4F41E0B201C3010E94E90E182F811145
:1024000025C09B81F201818198133CC09C8182810F
:10241000981338C0808182FF12C02394F2E02F16F7
:1024200009F48ECF83E0281609F496CF91E029169F
:1024300009F4CECE15E00AC082E094E0BFCFF401EB
:102440008387822D880F820D8F5F8083812F2D9649
:102450000FB6F894DEBF0FBECDBFDF91CF911F91B5
:102460000F91FF90EF90DF90CF90BF90AF909F9033
:102470008F907F906F905F904F903F902F90089536
:1024800011E0E4CF17E0E2CF4F925F926F927F921C
:102490008F929F92AF92CF92EF92FF920F931F93E2
:1024A000CF93DF9300D0CDB7DEB76A8341155105D6
:1024B000B9F1F9016081623098F149012A013C01CA
:1024C00040E86CE10E94D50E87E08983A12CC12CE5
:1024D000CE0101967C018401920141E0BE016E5F54
:1024E0007F4FC3010E94A410811109C0F4018081B3
:1024F0008230C1F481E09981911101C080E00F9098
:102500000F90DF91CF911F910F91FF90EF90CF909F
:10251000AF909F908F907F906F905F904F900895B5
:1025200084E0EDCF81E0EBCF9A01AB0166E20C9441
:1025300044120F931F93CF93DF9300D01F92CDB718
:10254000DEB78C0182E08B8340E064E2C8010E9428
:102550004B0E40E066E2C8010E944B0E46E268E482
:10256000C8010E944B0EAE014D5F5F4FBE016F5F11
:102570007F4FC8010E949412982F9D7F81E009F03F
:1025800080E00F900F900F90DF91CF911F910F91EE
:1025900008958F929F92AF92CF92EF92FF920F93F6
:1025A0001F93CF93DF9300D000D0CDB7DEB74C019F
:1025B00080E589831A829E012D5F3F4F42E0BE0174
:1025C0006F5F7F4FC4010E94E90E811116C0A12CDC
:1025D000C12CF12CE12C10E000E030E020E044E0E0
:1025E000BE016F5F7F4FC4010E94A410833021F0B1
:1025F000811103C081E001C080E00F900F900F9027
:102600000F90DF91CF911F910F91FF90EF90CF909E
:10261000AF909F908F90089548E060E10C94D50EA4
:102620001F920F920FB60F9211242F933F938F9307
:102630009F93AF93BF938091660490916704A0919C
:102640006804B09169043091650426E0230F2D37AA
:1026500068F129E8230F0396A11DB11D209365049D
:102660008093660490936704A0936804B093690410
:102670008091610490916204A0916304B09164041C
:102680000196A11DB11D8093610490936204A093F3
:102690006304B0936404BF91AF919F918F913F9178
:1026A0002F910F900FBE0F901F9018950296A11DAD
:1026B000B11DD4CF2FB7F894609166047091670470
:1026C00080916804909169042FBF08953FB7F894F2
:1026D0008091610490916204A0916304B0916404BC
:1026E00026B5A89B05C02F3F19F00196A11DB11D6D
:1026F0003FBFBA2FA92F982F8827BC01CD01620FA9
:10270000711D811D911D43E0660F771F881F991F62
:102710004A95D1F708958F929F92AF92BF92CF9230
:10272000DF92EF92FF926B017C010E9466134B01D6
:102730005C01C114D104E104F104E9F00E94C21764
:102740000E946613681979098A099B09683E7340DB
:102750008105910570F321E0C21AD108E108F10862
:1027600088EE880E83E0981EA11CB11CC114D10410
:10277000E104F10429F7FF90EF90DF90CF90BF9034
:10278000AF909F908F9008950000000083309105D6
:1027900028F0880F991F05970197F1F7089578940D
:1027A00084B5836084BD85B5836085BDEEE6F0E0C9
:1027B000808181608083E1E8F0E082E08083808135
:1027C00081608083E0E8F0E0808181608083E1EBDC
:1027D000F0E0808184608083E0EBF0E080818160C4
:1027E000808386E880937A001092C10008951F9339
:1027F000CF93DF93182FEB0161E00E947D142097A7
:1028000039F460E0812FDF91CF911F910C94B914BE
:10281000CF3FD10511F461E0F5CFE12FF0E0E859A9
:10282000FF4FE491E43031F140F4E230B1F0E330B5
:10283000E1F0C038D1057CF7E4CFE83029F1E93088
:1028400059F1E530B1F7809180008062809380007B
:10285000D0938B00C0938A0004C084B5806884BD87
:10286000C7BDDF91CF911F91089584B5806284BD6B
:10287000C8BDF7CF80918000806880938000D0939E
:102880008900C0938800EDCF8091B000806880936C
:10289000B000C093B300E5CF8091B0008062809318
:1028A000B000C093B400DDCF843081F028F48230D2
:1028B000E9F08330F9F00895883071F0893091F0B3
:1028C0008530B9F4809180008F7D03C080918000B5
:1028D0008F778093800008958091B0008F778093E8
:1028E000B00008958091B0008F7DF9CF84B58F77C7
:1028F00084BD089584B58F7DFBCFCF93DF9390E0A7
:10290000FC01E158FF4F24918A569F4FFC018491AE
:102910008823C9F090E0880F991FFC01EF53FF4F07
:10292000A591B491FC01E954FF4FC591D491611177
:102930000DC09FB7F8948C91209582238C93888149
:10294000282328839FBFDF91CF910895623051F4EF
:102950009FB7F8943C91822F809583238C93E881D4
:102960002E2BEFCF8FB7F894EC912E2B2C938FBF9B
:10297000EACF1F93CF93DF93282F30E0F901E85976
:10298000FF4F8491F901E158FF4FD491F901EA56C4
:10299000FF4FC491CC23A9F0162F81110E9454142B
:1029A000EC2FF0E0EE0FFF1FE954FF4FA591B4911B
:1029B0008FB7F894EC91111108C0D095DE23DC9309
:1029C0008FBFDF91CF911F910895DE2BF8CFCF936A
:1029D000DF93282F30E0F901E859FF4F8491F90186
:1029E000E158FF4FD491F901EA56FF4FC491CC232F
:1029F000A1F081110E945414EC2FF0E0EE0FFF1FA4
:102A0000E355FF4FA591B491EC91ED2381E090E067
:102A100009F480E0DF91CF91089580E090E0FACF53
:102A2000FC01918D228D892F90E0805C9F4F821B4D
:102A300091098F7399270895FC01918D828D9817C4
:102A400031F0828DE80FF11D858D90E008958FEFB4
:102A50009FEF0895FC01918D828D981761F0A28DF2
:102A6000AE0FBF2FB11D5D968C91928D9F5F9F73AE
:102A7000928F90E008958FEF9FEF0895FC01538DA2
:102A8000448D252F30E0842F90E0821B930B541748
:102A900010F0CF960895019708958DE896E1892B5F
:102AA00049F080E090E0892B29F00E948D16811179
:102AB0000C9400000895FC01A48DA80FB92FB11D3E
:102AC000A35ABF4F2C91848D90E001968F73992764
:102AD000848FA689B7892C93A089B1898C91806451
:102AE0008C93938D848D981306C00288F389E02D12
:102AF00080818F7D80830895CF93DF93EC01888D53
:102B00008823B9F0AA89BB89E889F9898C9185FD68
:102B100003C0808186FD0DC00FB607FCF7CF8C91F6
:102B200085FFF2CF808185FFEDCFCE010E945B153E
:102B3000E9CFDF91CF910895EF92FF920F931F930A
:102B4000CF93DF93EC0181E0888F9B8D8C8D981360
:102B500016C0E889F989808185FF11C0EE89FF8957
:102B60006083E889F98980818064808381E090E0D6
:102B7000DF91CF911F910F91FF90EF900895F62E66
:102B80000B8D10E00F5F1F4F0F731127E02E8C8D00
:102B90008E110CC00FB607FCFACFE889F989808145
:102BA00085FFF5CFCE010E945B15F1CFEB8DEC0FC9
:102BB000FD2FF11DE35AFF4FF0820B8FEA89FB894D
:102BC00080818062D2CFCF92DF92EF92FF921F93EB
:102BD000CF93DF93EC016A017B01122F60E874E868
:102BE0008EE190E0A70196010E94DF172150310984
:102BF000410951095695479537952795E889F989EF
:102C000082E08083211580E1380798F0E889F9890E
:102C1000108260E472E48FE090E0A70196010E94C8
:102C2000DF172150310941095109569547953795CC
:102C30002795EC85FD853083EE85FF852083188EF2
:102C4000EC89FD891083EA89FB898081886980830A
:102C5000EA89FB8980818F7D8083DF91CF911F91ED
:102C6000FF90EF90DF90CF9008951F920F920FB6D4
:102C70000F9211242F938F939F93EF93FF93E091E3
:102C80007A04F0917B048081E0918004F0918104CA
:102C900082FD1BC09081809183048F5F8F73209190
:102CA0008404821741F0E0918304F0E0E659FB4F81
:102CB000958F80938304FF91EF919F918F912F9136
:102CC0000F900FBE0F901F9018958081F4CF1F9228
:102CD0000F920FB60F9211242F933F934F935F9350
:102CE0006F937F938F939F93AF93BF93EF93FF93D4
:102CF0008AE694E00E945B15FF91EF91BF91AF913E
:102D00009F918F917F916F915F914F913F912F9103
:102D10000F900FBE0F901F9018958AE694E00E94C6
:102D2000101521E0892B09F420E0822F0895EAE6AE
:102D3000F4E01382128288EE93E0A0E0B0E0848396
:102D40009583A683B78381E392E09183808385ECAA
:102D500090E09587848784EC90E09787868780EC65
:102D600090E0918B808B81EC90E0938B828B82EC56
:102D700090E0958B848B86EC90E0978B868B118E00
:102D8000128E138E148E0895AF92BF92CF92DF925F
:102D9000EF92FF920F931F93CF93DF936C017B0110
:102DA0008B01040F151FEB015E01AE18BF08C017A1
:102DB000D10759F06991D601ED91FC910190F08114
:102DC000E02DC6010995892B79F7C501DF91CF91D7
:102DD0001F910F91FF90EF90DF90CF90BF90AF9039
:102DE0000895FB0101900020E9F73197AF01461BE0
:102DF000570BDC01ED91FC910280F381E02D0994E9
:102E00006115710511F00C94F11690E080E00895C1
:102E1000DC01ED91FC910190F081E02D09948F92FD
:102E20009F92AF92BF92EF92FF920F931F93CF9317
:102E3000DF93CDB7DEB7A1970FB6F894DEBF0FBE14
:102E4000CDBF7C01FA01CB0119A2223008F42AE09F
:102E50008E010F5D1F4F822E912CB12CA12CBF0132
:102E6000A50194010E94DF17F901CA016A300CF52F
:102E7000605DD8016E938D01232B242B252B79F7D0
:102E800090E080E0109721F0BD01C7010E94F1168B
:102E9000A1960FB6F894DEBF0FBECDBFDF91CF91E4
:102EA0001F910F91FF90EF90BF90AF909F908F90E8
:102EB0000895695CDECF2115310541F4DC01ED9107
:102EC000FC910190F081E02D642F09940C940F1770
:102ED0009A01462F50E070E060E00C945B174F922F
:102EE0005F926F927F92AF92BF92CF92DF92EF92FA
:102EF000FF920F931F93CF93DF93CDB7DEB72901D6
:102F00003A019B01AC012419350946095709898901
:102F10009A89AB89BC89BC01CD016A197B098C09EE
:102F20009D090E94C317A801970124193509460974
:102F300057090E940118CA01B9016A0D7B1D8C1D39
:102F40009D1DDF91CF911F910F91FF90EF90DF902A
:102F5000CF90BF90AF907F906F905F904F9008950B
:102F60000E94401808950E94CF130E94B2170E9439
:102F7000DB00CDE4D5E10E949C052097E1F30E949F
:102F80004D15F9CF0895DB018F939F930E9426186A
:102F9000BF91AF91A29F800D911DA39F900DB29FF5
:102FA000900D11240895991B79E004C0991F96177C
:102FB00008F0961B881F7A95C9F780950895A1E2BD
:102FC0001A2EAA1BBB1BFD010DC0AA1FBB1FEE1FA3
:102FD000FF1FA217B307E407F50720F0A21BB30BEE
:102FE000E40BF50B661F771F881F991F1A9469F76A
:102FF00060957095809590959B01AC01BD01CF01C6
:103000000895052E97FB1EF400940E94181857FD92
:1030100007D00E94DF1707FC03D04EF40C94181859
:1030200050954095309521953F4F4F4F5F4F0895F4
:1030300090958095709561957F4F8F4F9F4F089524
:10304000EE0FFF1F0590F491E02D09940E943118B6
:10305000A59F900DB49F900DA49F800D911D1124EC
:103060000895A29FB001B39FC001A39F700D811D61
:103070001124911DB29F700D811D1124911D089581
:1030800081E090E0F8940C945518FB01DC018D91DF
:10309000019080190110D9F3990B0895FB01DC010F
:0E30A00001900D920020E1F70895F894FFCF03
:1030AE008C01A601C001DA01050101781E274163DA
:1030BE006365737320436F64653F00000000008AF0
:1030CE0037F28041544347474354410000004000CB
:1030DE001400540041636365737300417574686F27
:1030EE0072697A65642100436F6E67726174756CE4
:1030FE006174696F6E73210044656E6965642100A9
:10310E0048656C70202D2050757A7A6C65200043CE
:10311E007573746F6D204D65737361676500000084
:10312E000000B017000000009700930048656C7017
:10313E00206D65737361676520666F722070757A96
:10314E007A6C6520340048656C70206D6573736110
:10315E00676520666F722070757A7A6C6520330011
:10316E0048656C70206D65737361676520666F725C
:10317E002070757A7A6C6520320048656C70206D0F
:10318E0065737361676520666F722070757A7A6CED
:10319E0065203100414354475F14071508000000B5
:1031AE00009700930000000000A307C416E906EC88
:1031BE0006000000006F089E08E90638080F081682
:1031CE0008290800000000C3109912B30D0000007A
:1031DE00009C15C4163E157C1510152A151C1500DD
:00000001FF
